:020000040000FA
:04000000CF303A289B
:08000800A000030EA100831209
:1000100005191128831601178312B2308100B0012F
:100020002C2883160113831203140B190310A80D37
:10003000A90DAA0DAB0DAC0DAC16FF302C02031DA3
:100040002C28FA302B02031D2C2831152A08AF006A
:100050002908AE002808AD008B100B11210E83007B
:06006000A00E200E0900B5
:0C007400203084008001840A80300402E7
:10008000031C3C28F22183160C308505870183125E
:10009000850187010730990000309A0010308316DF
:1000A0008E008312603083168F0083120030831617
:1000B00091009F008312C830831681008312313073
:1000C0009000003083168C00831210308B00BC1B14
:1000D0006F2885196F286400851D6B2827230A2344
:1000E00081018E018F010B118B100B108C018B176E
:1000F000872031199320B30B852803108519031429
:10010000B90DF030390203194E216D2378286400AF
:100110003210B00A301F9228AC01AB01AA01A9012C
:10012000A801B001080031110130B7008B13203055
:10013000370783169B001C141A088312A400103082
:10014000370783169B001C141A088312A300A6000D
:100150000230A6060030370783169B001C141A08CD
:100160008312A200A7000130A7068B17321CBE28FD
:1001700022090339A200A309A409A50924082F0212
:10018000031D482923082E02031D482922082D0299
:10019000031D482901303702031DD3283D18D328F9
:1001A0003D143E14142202303702031DDC28BD1812
:1001B000DC28BD143E14232203303702031DE5283A
:1001C0003D19E5283D153E142F2204303702031D4A
:1001D000EE28BD19EE28BD153E143B22053037022E
:1001E000031DF7283D1AF7283D163E144A22063013
:1001F0003702031D0029BD1A0029BD163E145922DD
:1002000007303702031D09293D1B09293D173E14FC
:10021000682208303702031D1229BD1B1229BD17A1
:100220003E14772209303702031D1B295E181B2953
:100230005E143E1482220A303702031D2429DE1880
:100240002429DE143E148D220B303702031D2D2984
:100250005E192D295E153E1498220C303702031DBD
:100260003629DE193629DE153E14A3220D30370259
:10027000031D3F295E1A3F295E163E14AE220E3042
:100280003702031D4829DE1A4829DE163E14B9221A
:10029000B70A0F3037020318080096280130B6005D
:1002A000B300B400B500B70085018701B113872002
:1002B000B30B9E29031085190314B90DF0303902D0
:1002C0000319C529B40B9E29013037020319C42232
:1002D000023037020319C922033037020319CE2234
:1002E000043037020319D322053037020319D8220C
:1002F000063037020319DD22073037020319E222E4
:10030000083037020319E722093037020319EC22BB
:100310000A3037020319F1220B3037020319F62293
:100320000C3037020319FB220D303702031900236A
:100330000E303702031905239630B400311D5729BA
:100340003111321CA8292D090339AD00AE09AF09BE
:100350002F1C57298E018F010C1C57290C102E1EA3
:1003600057298B1320303707BB002F08BA00DD2137
:1003700010303707BB002E08BA00DD2100303707E8
:10038000BB002D08BA00DD218B1785018701B70A54
:10039000B6010F303702031C57290A2308003E1C00
:1003A00008003E101030BB003D08BA00DD2130309F
:1003B000BB005E08BA00DD2108008B133A088316E3
:1003C0001C159A0083123B0883169B0055309D0034
:1003D000AA309D009C1464009C18EB291C11831208
:1003E0008B170800831600309B001C141A08831218
:1003F000BC00831610309B001C141A088312BD0029
:10040000831630309B001C141A088312DE00FF3064
:10041000C800CA15CB15CC15CD15CE15CF15D015E6
:10042000D115D215D31508008130BD05FF30DE058A
:100430000130C405C0000030C200C600BC185F1403
:10044000BC18DF1408008230BD05FF30DE05023025
:10045000C405C0000030C200C6005F100800843030
:10046000BD05FF30DE050630C405C0000030C20007
:10047000C6005F1008008830BD05FF30DE0509307A
:10048000C405C0000830C200C600BC185F14BC1808
:10049000DF1408009030BD05FF30DE051930C405BB
:1004A000C0000030C200C600BC185F14BC18DF14C6
:1004B0000800A030BD05FF30DE052130C405C000B6
:1004C0000030C200C600BC185F14BC18DF1408005E
:1004D000C030BD05FF30DE051030C405C00000305F
:1004E000C200C600BC185F14BC18DF140800FF303F
:1004F000BD05C030DE055030C505C1000030C30069
:10050000C70008007F30BD05C130DE052030C505BD
:10051000C1000030C300C70008007F30BD05C230F5
:10052000DE05E030C505C1002030C300C70008006B
:100530007F30BD05C430DE055030C505C100003038
:10054000C300C70008007F30BD05C830DE0550304D
:10055000C505C1000030C300C70008007F30BD05DD
:10056000D030DE055030C505C1000030C300C700E3
:1005700008007F30BD05E030DE054030C505C10014
:100580000030C300C7000800103085060030870621
:1005900008002030850600308706080021308506D7
:1005A00000308706080012308506003087060800F4
:1005B00012308506023087060800103085060430A8
:1005C00087060800003085060230870608000030E4
:1005D0008506113087060800003085062030870622
:1005E0000800003085063830870608000030850690
:1005F0001130870608000030850611308706080094
:100600000030850611308706080000308506393035
:10061000870608003D181422BD1823223D192F22F9
:10062000BD193B223D1A4A22BD1A59223D1B6822A0
:10063000BD1B77225E188222DE188D225E19982259
:10064000DE19A3225E1AAE22DE1AB9220800B60114
:10065000B301B4013C1C2F2BBC01BC14312BBC01D9
:100660003C143C08B6006400352B362B372B382B56
:10067000392BFF30B41B8500B41F8501B30B332B1E
:10068000B40B332B0310B60CB608031D332B00300C
:10069000BB003C08BA00DD21080005125C180516F5
:1006A000DC1C8512DC1885165C1D05105C19051410
:1006B000DC1D8510DC1985145C1E87105C1A8714FC
:1006C000DC1E0711DC1A07155C1F07105C1B0714E2
:1006D000DC1F8712DC1B871608008F08031908002F
:1006E0008F0178308E00C80F9F2DC80A441C9D2BA7
:1006F000461C8E2BCA1C7F2BCA014A15AB2B4A1DE8
:10070000842BCA01CA15AB2BCA1D892BCA014A16F4
:10071000AB2B4A1EAB2BCA01CA14AB2B4A1D932B21
:10072000CA014A16AB2BCA1D982BCA014A16AB2B1D
:100730004A1EAB2BCA01CA14AB2BCA1CA22BCA017E
:100740004A15AB2B4A1DA72BCA01CA15AB2B4A1E53
:10075000AB2BCA014A15C41CD22BC61CC32BCB1C05
:10076000B42BCB014B15E02B4B1DB92BCB01CB157B
:10077000E02BCB1DBE2BCB014B16E02B4B1EE02BF1
:10078000CB01CB14E02B4B1DC82BCB014B16E02B20
:10079000CB1DCD2BCB014B16E02B4B1EE02BCB0101
:1007A000CB14E02BCB1CD72BCB014B15E02B4B1DD7
:1007B000DC2BCB01CB15E02B4B1EE02BCB014B15DB
:1007C000441D072C461DF82BCC1CE92BCC014C15E5
:1007D000152C4C1DEE2BCC01CC15152CCC1DF32B60
:1007E000CC014C16152C4C1E152CCC01CC14152C00
:1007F0004C1DFD2BCC014C16152CCC1D022CCC0114
:100800004C16152C4C1E152CCC01CC14152CCC1CC4
:100810000C2CCC014C15152C4C1D112CCC01CC15DD
:10082000152C4C1E152CCC014C15C41D3D2CC61D81
:100830002E2CCD1C1F2CCD014D155F134B2C4D1DA7
:10084000242CCD01CD154B2CCD1D292CCD014D16C1
:100850004B2C4D1E4B2CCD01CD144B2C4D1D332C50
:10086000CD014D164B2CCD1D382CCD014D164B2CEA
:100870004D1E4B2CCD01CD144B2CCD1C422CCD014B
:100880004D154B2C4D1D472CCD01CD154B2C4D1E20
:100890004B2CCD014D155F1B742C441E742C461E31
:1008A000652CCE1C562CCE014E15822C4E1D5B2C79
:1008B000CE01CE15822CCE1D602CCE014E16822C80
:1008C0004E1E822CCE01CE14822C4E1D6A2CCE01DF
:1008D0004E16822CCE1D6F2CCE014E16822C4E1E33
:1008E000822CCE01CE14822CCE1C792CCE014E153A
:1008F000822C4E1D7E2CCE01CE15822C4E1E822CBB
:10090000CE014E15C41EA92CC61E9A2CCF1C8B2CB2
:10091000CF014F15B72C4F1D902CCF01CF15B72C01
:10092000CF1D952CCF014F16B72C4F1EB72CCF01E2
:10093000CF14B72C4F1D9F2CCF014F16B72CCF1DB6
:10094000A42CCF014F16B72C4F1EB72CCF01CF14BC
:10095000B72CCF1CAE2CCF014F15B72C4F1DB32C8D
:10096000CF01CF15B72C4F1EB72CCF014F15DF1875
:10097000E02C451EE02C471ED12CD01CC22CD001EF
:100980005015EE2C501DC72CD001D015EE2CD01DCB
:10099000CC2CD0015016EE2C501EEE2CD001D014D1
:1009A000EE2C501DD62CD0015016EE2CD01DDB2C79
:1009B000D0015016EE2C501EEE2CD001D014EE2C8F
:1009C000D01CE52CD0015015EE2C501DEA2CD00186
:1009D000D015EE2C501EEE2CD0015015DF18172D1F
:1009E000C51E172DC71E082DD11CF92CD10151157C
:1009F000252D511DFE2CD101D115252DD11D032DE5
:100A0000D1015116252D511E252DD101D114252D91
:100A1000511D0D2DD1015116252DD11D122DD101A4
:100A20005116252D511E252DD101D114252DD11C56
:100A30001C2DD1015115252D511D212DD101D1156F
:100A4000252D511E252DD1015115DF184F2D451F84
:100A50004F2D471F402DD21C312DD2015215DF13CF
:100A60005D2D521D362DD201D2155D2DD21D3B2D8F
:100A7000D20152165D2D521E5D2DD201D2145D2D74
:100A8000521D452DD20152165D2DD21D4A2DD20187
:100A900052165D2D521E5D2DD201D2145D2DD21C39
:100AA000542DD20152155D2D521D592DD201D21552
:100AB0005D2D521E5D2DD2015215DF18882DDF1BD2
:100AC000882DC51F882DC71F792DD31C6A2DD301F2
:100AD0005315962D531D6F2DD301D315962DD31D70
:100AE000742DD3015316962D531E962DD301D31476
:100AF000962D531D7E2DD3015316962DD31D832D78
:100B0000D3015316962D531E962DD301D314962D33
:100B1000D31C8D2DD3015315962D531D922DD3012A
:100B2000D315962D531E962DD3015315CF21400872
:100B3000C4004108C5005F18DF145F1CDF104808BF
:100B4000C9000C304A05031D05120C304B05031D6E
:100B500085120C304C05031D05100C304D05031D8E
:100B600085100C304E05031D87100C304F05031DFA
:100B700007110C305005031D07100C305105031DE3
:100B800087120C305205031D07120C305305031D4C
:100B9000871149080E020318F92D12304A05031D6A
:100BA000051612304B05031D851612304C05031D2A
:100BB000051412304D05031D851412304E05031D1A
:100BC000871412304F05031D071512305005031D01
:100BD000071412305105031D871612305205031DEC
:100BE000071612305305031D8715FF3048020319FD
:100BF00008008F08031D0800872049080E02031C07
:100C0000F92D18304A05031D051206304A05031D4B
:100C1000051618304B05031D851206304B05031DC4
:100C2000851618304C05031D051006304C05031DB4
:100C3000051418304D05031D851006304D05031DA4
:100C4000851418304E05031D871006304E05031D10
:100C5000871418304F05031D071106304F05031D7B
:100C6000071518305005031D071006305005031DE9
:100C7000071418305105031D871206305105031D56
:100C8000871618305205031D071206305205031D42
:100C9000071618305305031D871106305305031D31
:040CA00087150800AC
:084000000700030006000600A2
:02400E00CC33B1
:10420000010078007A007C007E007B0079007F004E
:104210007D007A0078007E007C007D007F007900C0
:104220000200F200F600FA00FE00F200F600FA00CA
:10423000FE00F200F600FA00FE00F200F600FA00BE
:10424000FF00050005000500050009000900090040
:1042500009000D000D000D000D00110011001100EE
:104260000100FF00FF00FF00FF00FF00FF00FF0054
:10427000FF00FF00FF00FF00FF00FF00FF00FF0046
:10428000FF007B00FF00FF00FF00FF00FF00FF00BA
:10429000FF00FF00FF00FF00FF00FF00FF00FF0026
:1042A000FF00FE00FF00FF00FF00FF00FF00FF0017
:1042B000FF00FF00FF00FF00FF00FF00FF00FF0006
:1042C000FF001100FF00FF00FF00FF00FF00FF00E4
:1042D000FF00FF00FF00FF00FF00FF00FF00FF00E6
:1042E000FF00FF00FF00FF00FF00FF00FF00FF00D6
:1042F000FF00FF00FF00FF00FF00FF00FF00DD00E8
:00000001FF
